:10000000C3C2FECFFDCFFCCFFBCFFACFF9CFF8CFE5
:10001000F7CFF6CFF5CFF4CFF3CFF2CFF1CFF0CFCC
:06002000EFCFEECFEDCFA3
:10058800BFE5BDBFB4E0BEBFCDB7DEB76197CDBF95
:10059800DEBF21962F923F924F925F92BEB5B16017
:1005A800BEBDBEB5B260BEBDBEB5B460BEBDB1EC29
:1005B800B7BBBEE3B8BBBCE3B4BBB3ECB5BBB3E8F5
:1005C800B1BBBCE7B2BB84DD99DEB1E02B2E24DEE3
:1005D800BCE02B2E21DEFE01B1E4B193B2E7B1936A
:1005E800BDE6B193B1E6B193B4E7B193B5E7B19382
:1005F800B2E7B193B1E6B193BDE2B193B5E7B19378
:10060800B2E7B193B1E6B193BCE6B193BEE2B19360
:10061800B2E7B193B5E7B193B0E0B1938E01280189
:10062800B1E03B2EB1E02B2EB6DD2DE01DE208ED4A
:100638000A95F1F71A95E1F72A95D1F7000000001D
:10064800222433244BDE00938300B1E02B2EB0E04C
:100658003B2E44DE00938200B2E02B2EB0E03B2E0E
:100668003DDE00936E00B3E02B2EB0E03B2E36DE6D
:1006780000936D00B4E02B2EB0E03B2E2FDE0093EC
:100688006C00B5E02B2EB0E03B2E28DE00936B000B
:10069800B6E02B2EB0E03B2E21DE00937000B7E0D1
:1006A8002B2EB0E03B2E1ADE00936F00B8E02B2E05
:1006B800B0E03B2E13DE0093710020916D00309165
:1006C8006E00009182001091830020173107D9F441
:1006D800B8ECB0936D00B0E0B0936E00B0E5B093A5
:1006E8008200B0E0B0938300B6E4B0936B00B0E052
:1006F800B0936C00BCEDB0936F00B0E0B0937000A5
:10070800B4E6B0937100B0B3B2FDF3C1B1E02B2EE3
:1007180083DDFE01B5E7B193B3E7B193B4E7B193D5
:10072800B1E6B193B6E7B193BBE6B193B1E6B19345
:10073800BFE5B193BDE6B193B9E6B193BEE6B19317
:10074800B0E0B1938E012801B1E03B2EB1E02B2E31
:1007580022DDB0B3B2FFFDCFB0B3B2FF33C0B0B348
:10076800B3FD0DC000918200109183000F5F1F4FF1
:100778000093820010938300B0B3B3FFFDCFB0B3F2
:10078800B4FD0DC00091820010918300015010400B
:100798000093820010938300B0B3B4FFFDCFB0E69E
:1007A8004B2EB0E05B2E2090820030908300BDDE9F
:1007B800B0E64B2EB0E05B2EB1E03B2EB2E02B2E24
:1007C800EADCCACFB0B3B2FFFDCFB1E02B2E24DDF7
:1007D800FE01B5E7B193B3E7B193B4E7B193B1E6DE
:1007E800B193B6E7B193BBE6B193B1E6B193BFE578
:1007F800B193BDE6B193B1E6B193B8E7B193B0E078
:10080800B1938E012801B1E03B2EB1E02B2EC3DC61
:10081800B0B3B2FF33C0B0B3B3FD0DC000916D00EB
:1008280010916E000F5F1F4F00936D0010936E00C4
:10083800B0B3B3FFFDCFB0B3B4FD0DC000916D00F0
:1008480010916E000150104000936D0010936E00DF
:10085800B0B3B4FFFDCFB0E64B2EB0E05B2E2090D6
:100868006D0030906E0061DEB0E64B2EB0E05B2E7E
:10087800B1E03B2EB2E02B2E8EDCCACFB0B3B2FF74
:10088800FDCFB1E02B2EC8DCFE01B4E7B193B8E68A
:10089800B193B3E6B193BFE5B193BFE6B193BEE6BA
:1008A800B193BFE5B193BDE6B193B9E6B193BEE6A6
:1008B800B193B0E0B1938E012801B1E03B2EB1E0D5
:1008C8002B2E69DCB0B3B2FF33C0B0B3B3FD0DC09B
:1008D80000916B0010916C000F5F1F4F00936B002D
:1008E80010936C00B0B3B3FFFDCFB0B3B4FD0DC02F
:1008F80000916B0010916C000150104000936B0048
:1009080010936C00B0B3B4FFFDCFB0E64B2EB0E04F
:100918005B2E20906B0030906C0007DEB0E64B2E0B
:10092800B0E05B2EB1E03B2EB2E02B2E34DCCACF18
:10093800B0B3B2FFFDCFB1E02B2E6EDCFE01B4E701
:10094800B193B8E6B193B3E6B193BFE5B193BFE60F
:10095800B193BEE6B193BFE5B193BDE6B193B1E6FD
:10096800B193B8E7B193B0E0B1938E012801B1E03B
:100978003B2EB1E02B2E0FDCB0B3B2FF33C0B0B3C7
:10098800B3FD0DC000916F00109170000F5F1F4FF5
:1009980000936F0010937000B0B3B3FFFDCFB0B3F6
:1009A800B4FD0DC000916F0010917000015010400F
:1009B80000936F0010937000B0B3B4FFFDCFB0E6A2
:1009C8004B2EB0E05B2E20906F0030907000ADDDB4
:1009D800B0E64B2EB0E05B2EB1E03B2EB2E02B2E02
:1009E800DADBCACFB0B3B2FFFDCFB1E02B2E14DCF7
:1009F800FE01B4E7B193B8E6B193B3E6B193BFE5AE
:100A0800B193B4E7B193B9E6B193BDE6B193B5E656
:100A1800B193B0E0B1938E012801B1E03B2EB1E073
:100A28002B2EB9DBB0B3B2FF27C0B0B3B3FD08C0FB
:100A3800009171000F5F00937100B0B3B3FFFDCF59
:100A4800B0B3B4FD08C0009171000150009371006B
:100A5800B0B3B4FFFDCFB6E63B2EB0E04B2E2090EE
:100A6800710041DBB6E64B2EB0E05B2EB1E03B2EC9
:100A7800B2E02B2E90DBD6CF409083002224332483
:100A880055DB40908200B1E02B2EB0E03B2E4EDBD0
:100A980040906E00B2E02B2EB0E03B2E47DB40903A
:100AA8006D00B3E02B2EB0E03B2E40DB40906C0095
:100AB800B4E02B2EB0E03B2E39DB40906B00B5E064
:100AC8002B2EB0E03B2E32DB40907000B6E02B2E90
:100AD800B0E03B2E2BDB40906F00B7E02B2EB0E050
:100AE8003B2E24DB40907100B8E02B2EB0E03B2E6B
:100AF8001DDBB1E02B2E90DBB0E0BDBDB0E0BCBD8E
:100B0800B0E0B0936A0010916A000091710001177B
:100B1800E0F01BE003E60A95F1F71A95E1F7B0B3A8
:100B2800B6FD04C0B2B3B068B2BB03C0B2B3BF77FE
:100B3800B2BB10916A0000917100101731F000915A
:100B48006A000F5F00936A00DECF0CB5009378004F
:100B58000DB500937900B1E02B2EFADA00937600F8
:100B68001093770098012E5F3F4F40917A00509183
:100B78007B0024173507B0E008F4BFEF2B2F025095
:100B880010404017510700E008F40FEF022B41F026
:100B9800009176001091770000937A0010937B0003
:100BA8000090820010908300B0E000916D001091D9
:100BB8006E0020E0322F001911092B0B3B0B4091DE
:100BC8007A0050917B0060E0762FC7DABAE0A8017E
:100BD800B9017695679557954795BA95D1F70091DC
:100BE80082001091830020E0322F040F151F261F6A
:100BF800371F00937E0010937F002093800030936E
:100C0800810000937C0010937D00B0E64B2EB0E08D
:100C18005B2E18018ADCB0B3B2FD07C06FDBBCE005
:100C28002B2EFADAB1E02B2EF7DA00917500102F8F
:100C38001F5F1093750004E1011730F4B0E0B09322
:100C48007500B1E02B2EE8DAB0E64B2EB0E05B2E53
:100C5800BCE03B2EB2E02B2E9EDAB0E64B2EB0E085
:100C68005B2E20907800309079005FDCB0E64B2E48
:100C7800B0E05B2EBCE03B2EB1E02B2E8CDAB0B39B
:100C8800B6FD1CC0B2B3B068B2BBFE01BDE2B19301
:100C9800B4E5B193BFE6B193B5E7B193B3E6B193C9
:100CA800B8E6B193BDE2B193B0E0B1938E012801EB
:100CB800B5E03B2EB1E02B2E6EDA1BC0B2B3BF7786
:100CC800B2BBFE01B0E2B193B0E2B193B0E2B1932E
:100CD800B0E2B193B0E2B193B0E2B193B0E2B193B4
:100CE800B0E0B1938E012801B5E03B2EB1E02B2E88
:100CF80052DA309178004091790000916F0010919C
:100D080070003017410720E008F42FEF00916B00C6
:100D180010916C0003171407B0E008F4BFEF0B2F15
:100D2800022309F47CC0BFE4B883BEE4B983B0E20F
:100D3800BA83B0E0BB838E012801B1E03B2EB1E05D
:100D48002B2E29DAB8B3B160B8BB20917800309166
:100D5800790000917C0010917D0020173107C1F4C3
:100D6800B8B3BF7BB8BBB8B3BF77B8BBFE01BFE4AD
:100D7800B193BBE4B193B0E2B193B0E2B193B0E008
:100D8800B1938E012801B1E03B2EB2E02B2E03DA9D
:100D9800209178003091790000917C0010917D00BD
:100DA80002171307C0F4B8B3B064B8BBB8B3BF77C1
:100DB800B8BBFE01B4E4B193BFE4B193B7E5B19316
:100DC800BEE4B193B0E0B1938E012801B1E03B2EAF
:100DD800B2E02B2EE0D92091780030917900009173
:100DE8007C0010917D0020173107C0F4B8B3BF7B99
:100DF800B8BBB8B3B068B8BBFE01B5E5B193B0E510
:100E0800B193B0E2B193B0E2B193B0E0B1938E0187
:100E18002801B1E03B2EB2E02B2EBDD92AC0BFE499
:100E2800B883B6E4B983B6E4BA83B0E0BB838E0175
:100E38002801B1E03B2EB1E02B2EADD9B8B3BE7F6F
:100E4800B8BBB8B3BF7BB8BBB8B3BF77B8BBFE01FC
:100E5800B0E2B193B0E2B193B0E2B193B0E2B19332
:100E6800B0E0B1938E012801B1E03B2EB2E02B2E09
:0E0E780092D942CE5F904F903F902F90FFCFC7
:1000D800BBE3B0937300B0E0B0937400B7E8B6B96F
:0600E800B0E0B7B9089575
:10030400B0913500B77FB0933500B0913500BB7F15
:10031400B0933500B0913200BD7FB0933200B091FC
:100324003200BE7FB0933200B0913500BF7DB093F0
:100334003500B0913500BF7EB0933500B0913400E4
:10034400B860B0933400B0913400B460B09334001A
:10035400B0913400B061B0933400B0913400B06215
:10036400B0933400B0913100B160B0933100B091DA
:100374003100B260B09331009EDE9DDE9CDEB09110
:100384003500B062B0933500B0913500B061B093E0
:100394003500B0913500B860B093350095DEB0916A
:1003A4003500B77FB093350086DEB0913500B86074
:1003B400B093350089DEB0913500B77FB093350036
:1003C4007ADEB0913500B860B09335007DDEB0912F
:1003D4003500B77FB09335006EDEB0913500BF7E37
:1003E400B0933500B0913500B860B09335006CDE41
:1003F400B0913500B77FB09335005DDEB091350024
:10040400B860B093350060DEB0913500B77FB0932B
:100414003500B0913500BF7DB0933500B091320006
:10042400B260B0933200B0913500B860B09335003B
:100434004BDEB0913500B77FB09335003CDEB09110
:100444003200BD7FB0933200B0913500B061B093FB
:100454003500B0913500B860B093350035DEB09109
:100464003500B77FB0933500B0913500BF7EB093AF
:100474003500B0913500B860B093350025DEB091F9
:100484003500B77FB093350016DEB0913500B86003
:10049400B093350019DEB0913500B77FB0933500C5
:1004A400B0913500B061B0933500B0913500B860BB
:1004B400B093350009DEB0913500B77FB0933500B5
:1004C400FADDB0913500BF7EB0933500B0913500B0
:1004D400B860B0933500F8DDB0913500B77FB093C4
:1004E4003500B0913200B260B0933200B091320066
:1004F400B160B0933200B0913500B062B093350072
:10050400B0913500B061B0933500B0913500B8605A
:10051400B0933500D9DDB0913500B77FB093350085
:0E052400CADDB0917200B160B093720008950C
:1000BA001AE303E20A95F1F71A95E1F70000000046
:0200CA00089597
:0C00CC0002E00A95F1F700000000089522
:1002200027FAB0913200B1F9B093320026FAB091BA
:100230003200B0F9B093320025FAB0913500B5F92B
:10024000B093350024FAB0913500B4F9B09335007D
:10025000B091720000903500E894B0FF689402F805
:1002600000923500B0913500B860B09335002EDFB4
:10027000B0913500B77FB093350023FAB0913200CA
:10028000B1F9B093320022FAB0913200B0F9B093D4
:10029000320021FAB0913500B5F9B093350020FA5B
:1002A000B0913500B4F9B0933500B0917200009070
:1002B0003500E894B0FF689402F800923500B091E0
:1002C0003500B860B093350001DFB0913500B77FDD
:1002D000B0933500B0917200B0FF02C0EEDE01C0F5
:0402E000B1DE0895EE
:0A00440005E80A95F1F700000895A1
:10019E002F92B1E02B1619F4B0E82B2E14C0B2E05A
:1001AE002B1619F4B0EC2B2E0EC0B3E02B1619F44F
:1001BE00B4E92B2E08C0B4E02B1619F4B4ED2B2E97
:1001CE0002C0B0E82B2E032D0150020D202E202E42
:1001DE0020D0B0917200BE7FB09372009201F901EF
:1001EE000081002379F0F90100813F932F932F9224
:1001FE00202E15DF2F902F913F9189010F5F1F4FFA
:10020E009801EDCFB0917200B160B09372002F9053
:02021E00089541
:10002C00B0917200BE7FB0937200F4D0B0917200A8
:08003C00B160B0937200089559
:1002E4000FB6BCB3B1FF02C00000FBCFF8943FBA15
:1002F4002EBABCB3B160BCBB0FBE1DB3012F0895B1
:00030400F9
:10053200F201B0E2B193B0E2B193B0E2B193B0E2B2
:10054200B193B0E3B193B0E0B19382010C5F1F4F5E
:100552009801B0E03B1611F4B0E02B1699F04AE096
:1005620050E0810173DD8D01005DF90100834AE0F5
:1005720050E081016BDD8C011801890101501040AE
:060582009801E7CF089587
:10004E00C801BA01AA1BBB1B51E107C0AA1FBB1FE7
:10005E00A617B70710F0A61BB70B881F991F5A9546
:08006E00A9F780959095089513
:1000EE00E32DF42DB0E2B193B0E2B193B0E3B1934E
:1000FE00B0E0B193032D142D0E5F1F4F9801B0E0A9
:10010E002B1681F04AE0022DC5DF092F005DF901A3
:10011E0000834AE0022DBEDF202E890101501040DF
:06012E009801EDCF0895D9
:1000A200992779E004C0991F941708F0941B001F48
:0800B2007A95C9F70095089545
:100134000FB6BCB3B1FF02C00000FBCFF8943FBAC6
:100144002EBA4DBABCB3B460BCBBBCB3B260BCBBCA
:040154000FBE08953D
:0A015800BFDF8DDF980189010895D3
:1000760007B1007E022907B9B6B1B064B6B9B6B108
:10008600B6FF02C00000FBCF24B130E005B1102F4F
:0C0096000027022B132B9801890108950C
:10016200049FD001159FF001249FE00DF11D069F11
:10017200E00DF11D349FF00D259FF00D169FF00D3F
:10018200079FF00D3327149FB00DE11DF31F059F4C
:0C019200B00DE11DF31F8D019F010895C9
:00000001FF
